:03200000022100BA
:03202B00022FF28F
:1021000075BF0143B70843B70453B6F743B6047924
:1021100000780AD9FED8FC785643B602D8FEE5B658
:1021200030E0F475BB9853B70F43B7A053B7FB43E8
:10213000B7027864D8FEE5B730E0DC53B7F775BF77
:102140000078FFE4F6D8FD90F0007F007E06E4F012
:10215000A3DFFCDEFA75819F0221960221DBE49366
:10216000A3F8E493A34003F68001F208DFF480298A
:10217000E493A3F85407240CC8C333C4540F442079
:10218000C8834004F456800146F6DFE4800B010268
:10219000040810204080902A3BE47E019360BCA399
:1021A000FF543F30E509541FFEE493A360010ECFB6
:1021B00054C025E060A840B8E493A3FAE493A3F8E0
:1021C000E493A3C8C582C8CAC583CAF0A3C8C582A0
:1021D000C8CAC583CADFE9DEE780BEAEB4EE7002CE
:1021E0007F01122B66E4F5BF7581C0D280D2B67D27
:1021F00002FF123F7F7B017AF079EE123BFC90F1F7
:1022000016EEF0A3EFF07B017AF079541235B0129C
:1022100030F9122E591242A1122ED380F27C0112F3
:102220002DA17F027E002202256FE86480F8E93349
:10223000E83360110460F0ED33EC337009E8FCE939
:10224000FDEAFEEBFF220460DED3EB9FEA9EE99DF0
:10225000E8C2E78CF0C2F795F0400CE8CCF8E9CD85
:10226000F9EACEFAEBCFFB12253A85D0F05804708C
:102270000320D5B3E80470075002B2D50225799245
:10228000D5EC0460F7E4CCC0E0C398F8603B941848
:102290006008400DD0E0FB022551E4FBFAC9FC8048
:1022A00028E830E406E4C9FBE4CAFCE830E305E4CE
:1022B000C9CACBFCE854076010F8C3E913F9EA1364
:1022C000FAEB13FBEC13FCD8F130F52FC3E49CFCC4
:1022D000EF9BFFEE9AFEED99FDD0E0FBEF4E4D4CEB
:1022E000701222DB03022576EC2CFCEF33FFEE3379
:1022F000FEED33FDED30E7EB022551EF2BFFEE3A1B
:10230000FEED39FDD0E0FB50130BBB000302257935
:10231000ED13FDEE13FEEF13FFEC13FC022551EC61
:102320004D6011E8497017ED33EC3304600DE4FCA7
:10233000FFFEFD22E933E8330470F802256F122511
:102340003A58046009E4CC2481500628500902253B
:1023500079284003022576C0E0EB4A7044B9800634
:10236000D0E0FB022565EF4E701CBD8008EBFFEA54
:10237000FEE9FD80EBE98DF0A4FEE5F0022408E91A
:10238000CDF9EAFEEBFFEF89F0A4FCE5F0CE89F091
:10239000A42EFFE435F0CD89F0A42DFEE435F080C5
:1023A00067EF4E7005BD80D780C3EF8BF0A4ACF013
:1023B000EE8BF0A42CFCE435F0F8EF8AF0A42CE5C9
:1023C000F038FCE433CB8DF0A42CFCE5F03BF8EEC8
:1023D0008AF0A42CFCE5F038F8E433CF89F0A42C83
:1023E000FCE5F038CF3400CE89F0A42FFFE5F03EB5
:1023F000FEE433C98DF0A42EFEE5F039CD8AF0A4B9
:102400002FFFE5F03EFEE43DFD33D0E0FB50070B2F
:10241000BB000F022579EC2CFCEF33FFEE33FEED11
:1024200033FD022551022579EC5D046005E859046D
:10243000700302256F12253A580460F6EC4860F2EA
:10244000EC7004FDFEFF22C860DB2481C85009C384
:1024500098600250060225769850CAF582E9294B09
:102460004A7005AB8202256575F0007C1A7880C33E
:10247000EF9BEE9AED99400DC3EF9BFFEE9AFEEDB8
:1024800099FDE842F0DC23ACF0D0E0FFD0E0FED0D4
:10249000E0FDAB8220E7101BEB60BAEC2CFCEF33C5
:1024A000FFEE33FEED33FD022551E803F830E7057A
:1024B000C0F075F000EF2FFFEE33FEED33FD40B8B6
:1024C00030E7C280AA75F020800E75F01080057587
:1024D000F0087D007E007F003392D530D5031226B0
:1024E000BBEC334010EF33FFEE33FEED33FDEC3346
:1024F000FCD5F0ED22E5F0247EA2D513CC92E7CDF9
:10250000CEFF22EDD2E7CD33EC3392D524814006C5
:10251000E4FFFEFDFC22FCE4CFCECDCC24E0501144
:1025200074FF80EDC3CC13CCCD13CDCE13CECF131F
:10253000CF0470F030D5DE0226BBE9D2E7C933E81C
:1025400033F892D5EDD2E7CD33EC33FC5002B2D55F
:1025500022EC30E7100FBF000C0EBE00080DBD00CE
:10256000040BEB6014A2D5EB13FCED92E7FD227493
:10257000FFFCFDFEFF22E480F8A2D574FF13FC7D72
:1025800080E480EFBB010689828A83E0225002E763
:1025900022BBFE02E32289828A83E49322BB010CE0
:1025A000E58229F582E5833AF583E0225006E925A4
:1025B00082F8E622BBFE06E92582F8E222E58229BE
:1025C000F582E5833AF583E49322BB010FF8E582B7
:1025D00029F582E5833AF583E028F0225009C58287
:1025E00029F8E58226F622BBFE09C58229F8E225F4
:1025F00082F222F8EA2583F583E9932822BB0106BB
:1026000089828A83F0225002F722BBFE01F322F86E
:10261000BB010DE58229F582E5833AF583E8F022D6
:102620005006E92582C8F622BBFE05E92582C8F2DC
:1026300022BC000BBE0029EF8DF084FFADF022E438
:10264000CCF875F008EF2FFFEE33FEEC33FCEE9D77
:10265000EC984005FCEE9DFE0FD5F0E9E4CEFD229E
:10266000EDF8F5F0EE8420D21CFEADF075F008EF29
:102670002FFFED33FD4007985006D5F0F222C398A6
:10268000FD0FD5F0EA22A3F8E0C5F025F0F0E582D1
:10269000158270021583E0C838F0E822BB010A8970
:1026A000828A83F0E5F0A3F0225006F709A7F0191B
:1026B00022BBFE06F3E5F009F31922C3E49FFFE411
:1026C0009EFEE49DFDE49CFC22EB9FF5F0EA9E4219
:1026D000F0E99D42F0EC6480C864809845F022EBFC
:1026E0009FF5F0EA9E42F0E99D42F0E89C45F02219
:1026F000E8600FECC313FCED13FDEE13FEEF13FFC8
:10270000D8F122E8600FEFC333FFEE33FEED33FD67
:10271000EC33FCD8F122BB010789828A83022A1399
:102720005005E9F8022A07BBFE05E9F8022A1F89CD
:10273000828A83022A2BECF0A3EDF0A3EEF0A3EF44
:10274000F022A8828583F0D083D0821227591227E5
:1027500059122759122759E473E493A3C583C5F08E
:10276000C583C8C582C8F0A3C583C5F0C583C8C5E5
:1027700082C822E3F5F009E208B5F06BDFF5806767
:10278000E3F5F009E608B5F05EDFF5805A87F00959
:10279000E608B5F052DFF6804E87F009E208B5F0A2
:1027A00046DFF6804288828C8387F009E0A3B5F08B
:1027B00036DFF6803288828C8387F009E493A3B5F4
:1027C000F025DFF5802188828C83E3F5F009E0A312
:1027D000B5F014DFF5801088828C83E3F5F009E40E
:1027E00093A3B5F002DFF402289E808780E98090F1
:1027F00080D4803C8015806C807C809D80B7808DEB
:1028000080A3804F8072803A0228AA89828A8363DB
:10281000A20188828C8363A201E493F5F0A363A2F2
:1028200001E493A363A201B5F074DFEDDEEB806EEB
:1028300089828A83E493F5F0A3E208B5F060DFF4BF
:10284000805C89828A83E0F5F0A3E608B5F04FDF6B
:10285000F5804B89828A83E0F5F0A3E208B5F03E6B
:10286000DFF5803A89828A83E493F5F0A3E608B520
:10287000F02CDFF480288002805389828A8363A24F
:102880000188828C8363A201E493F5F0A363A20123
:10289000E0A363A201B5F006DFEEDEEC80007FFF6F
:1028A000B5F0020F2240027F012289828A8363A24F
:1028B0000188828C8363A201E0F5F0A363A201E0AA
:1028C000A363A201B5F0D7DFEFDEED80D189828A64
:1028D0008363A20188828C8363A201E0F5F0A36385
:1028E000A201E493A363A201B5F0B3DFEEDEEC80B6
:1028F000AD88F0EF60010E4E60AFED2402B404002D
:10290000509CF582EB2402B40400509223234582AC
:10291000239027EA73E709F608DFFA8046E709F211
:1029200008DFFA803E88828C83E709F0A3DFFA8013
:1029300032E309F608DFFA8076E309F208DFFA806D
:102940006E88828C83E309F0A3DFFA806289828A31
:1029500083E0A3F608DFFA805689828A83E0A3F237
:1029600008DFFA804A80D280FA80C680D4806580F1
:10297000F28031801080A680EA809A80A880DA8078
:10298000E280CA803189828A8363A20188828C8333
:1029900063A201E493A363A201F0A363A201DFF3A6
:1029A000DEF1800B89828A83E493A3F608DFF9ECD9
:1029B000FAA9F0EDFB2289828A8363A20188828CC6
:1029C0008363A201E0A363A201F0A363A201DFF489
:1029D000DEF280DB89828A83E493A3F208DFF98048
:1029E000CE88F0EF60010E4E60C588F0ED2402B491
:1029F000040050BBF582EB2402B4040050B1232341
:102A000045822390296573E6FC08E6FD08E6FE088A
:102A1000E6FF22E0FCA3E0FDA3E0FEA3E0FF22E24C
:102A2000FC08E2FD08E2FE08E2FF22E493FC7401E8
:102A300093FD740293FE740393FF2258F00000008C
:102A40000000000000000000000000000000000086
:102A500000000000000044F0470000000042F03C8D
:102A60000000C100C10142F03A03E848F03E000016
:102A700000000000000048F04B00000000000000D3
:102A80000048F021000000000000000048F0540061
:102A90000101000000000048F029000000000000D3
:102AA000000050F06D000000000000000000000079
:102AB000000000000050F05D000000000000000079
:102AC000000000000000000048F0190000000000B5
:102AD00000000048F032000000000000000041F05B
:102AE000310050F07E0000000000000000000000F7
:102AF000000000000041F0460041F0180041F07D68
:102B000000C102C10341F05C0041F0530048F0E60F
:102B10000000000000000000008E198F188C1C8D32
:102B20001BE4F51DF51EF51FC0D0C0E0C0F043D07A
:102B30001812DFF94008D0F0D0E0D0D0D322D0F086
:102B4000D0E0D0D0C3228F18C0D0C0E0C0F043D0B6
:102B50001812DFF64008D0F0D0E0D0D0D322D0F069
:102B6000D0E0D0D0C32275BF0175BA10E4F5BFB173
:102B7000B1123FF8D12E12400A7189F1DFE4F5B8A5
:102B8000F5B9F5F8F5F9D2AF2275DA0075D9717596
:102B9000DC01E5DC30E00553D8FE80F675DA00751F
:102BA000D98075DB4975D815E5D820E1FB75D804C7
:102BB000D125E5D820E1FBD125E5D820E1FB75DB67
:102BC0004B75DC3A75D835E5D820E1FB75DD6075CD
:102BD000D845E5D820E1FBE4F5DBF5DCF5DD75D87B
:102BE00071E5D820E1FB75DA0075D9C075DB417558
:102BF000D815E5D820E1FB75B2024390024391025B
:102C0000E4F5B2439102F5DA75D9717F02FE7D08D1
:102C100012221D7D0512221D7D0612221D7D071226
:102C2000221D7D0912221D7D0A12221D7D0B1222FA
:102C30001D7D0C12221D7D0D7C01B1A175DA04757C
:102C4000D92FD11EB1997F037E007D007CE0B18138
:102C5000D10CB19B7F007E05B18AB1FE75D937D109
:102C600015B19B7F01B17BD10CB19B7F007E06B17A
:102C70008AB1FE75D93FD11EB1997F02B17BD10CCB
:102C8000B19B7F007E07B18AB1FE75D947D115B1DE
:102C90009B7F027E007D007CF1B181D10CB19B7FD6
:102CA000007E08B18AB1FE75D94FD115B19B7FF076
:102CB0007EFF7DFF7CFFB181D10CB19B7F007E093F
:102CC000B18AB1FE75D957D115B19B7F027E007DC7
:102CD000007CF4B181D10CB19B7F007E0AB18AB136
:102CE000FE75D95FD11EB1997F04B17BD10CB19B28
:102CF0007F007E0BB18AB1FE75D967D115B19B7F7C
:102D000003B17BD10CB19B7F007E0CB18AB1FE7503
:102D1000D96FD11EB1997F017E007D007CF4B18115
:102D20007FFF7EFF7DFF7C1FB19B7F007E0DB18A00
:102D30007F007E007D007C08B15475DA0075D98073
:102D4000E4F5D8E5D820E1FB53DBBE75D811E5D812
:102D500020E1FB2290F0AC12273690F0AFE0F5DBDB
:102D600090F0AEE0F5DC90F0ADE0F5DD90F0ACE099
:102D7000F5DE75D8F1E5D820E1FB227E007D007CF0
:102D8000F5B15475D8087F007E007D007C00B154F9
:102D900075D8087F007E007D007C00B15475D8088E
:102DA00022B15475DC01E5DC30E00553D8FE80F635
:102DB0002275B20375800875B2017580FE7586EFC5
:102DC000E4F5B275860D75800C75B203F59075B299
:102DD000017590DF7591BFF5B275916075B203759D
:102DE000B03C75B20175B03F75B1FCF5B275B1FC80
:102DF00075B201F5C875C908F5B275C908227F001A
:102E00007E007D007C08B15475DA04227FFF7EFFCE
:102E10007DFF7C3F227F007E007DA87C0E227F000C
:102E20007E007DA022E4F5DBF5DC75D83522D14C9F
:102E300075BCDB43BB0443BB03538FFE75BF0175F9
:102E4000BBABF5BF22D14C53BBFB80ED75BF017509
:102E5000BB9BE4F5BF438F012290F090743FF0C21A
:102E6000AFE5D820E1FBC0D9C0DAC0DBC0DCC0DDF3
:102E7000C0DE75BF80D1CCE4F5D8E5D820E1FB9069
:102E8000F08EE5DBF0A3E5DCF090F08EE030E502BB
:102E9000718990F08EE0FF5407600690F0907438CE
:102EA000F0D1CC90F090E05FF4F5DB90F08FE0F49F
:102EB000F5DC75D831E5D820E1FB75BFC0D0DED098
:102EC000DDD0DCD0DBD0DAD0D9D2AF2275DA007514
:102ED000D981227F05123885EF7002E188F1E37F06
:102EE00005F1EA90F0A5F090F099E090F0A4F09050
:102EF000F09AE090F0A3F090F09BE090F0A2F090B8
:102F0000F09CE090F0A9F090F09DE090F0A8F09097
:102F1000F09EE090F0A7F090F09FE090F0A6F07F98
:102F20000512384FC2AFC2C2D14590F0A2E064AAE8
:102F3000700FA3E064AA70097D017F5512399A8051
:102F40007990F0A2E06433703FA3E064337039F508
:102F5000BFF5BCFD7C03FFFE7119F189E4FFEFC3EF
:102F6000942074809480500974802FF8E4F60F80C8
:102F7000ED7880761175836FE4F5827F807146F17C
:102F8000897D047F5512399A22538FFEE4F5BFFFE5
:102F9000EFC39432748094805020E4FEEEF1D75059
:102FA00016E4FDEDF1D7500CE5BC30E20453BCFB58
:102FB000220D80EF0E80E50F80D675BF0175BB9B9B
:102FC000438F0143BB0475BCFF43BB03538FFE75A6
:102FD000BBABE4F5BF80FEC394FF748094802243B2
:102FE000A820227B017AF0798E221233EC90F0989F
:102FF000E022C0E0C0F0C083C082C0D075D00063C2
:10300000A201C083C08263A201C000C001C002C08F
:1030100003C004C005C006C00790F0DB743FF0E5B4
:10302000D820E1FBC0D9C0DAC0DBC0DCC0DDC0DE27
:1030300075BF8030C704C2C711BEE5B65401604AEF
:1030400053B6FE122ECC75D800E5D820E1FBAFDBDD
:10305000AEDCEF30E51B30E70A90F05C7480F0EFF7
:10306000547FFFEF30E60A90F05C7440F0EF54BFFD
:10307000FF122ECC90F0DBE05FF4F5DBAF06EEF450
:10308000F5DC75D831E5D820E1FB75BFC0D0DED0C6
:10309000DDD0DCD0DBD0DAD0D9D007D006D005D057
:1030A00004D003D002D001D00063A201D082D0832B
:1030B00063A201D0D0D082D083D0F0D0E0323000F3
:1030C0002490F03DE004F0700690F03CE004F090B5
:1030D000F03A11F290F03DE09F90F03CE09E400C01
:1030E000C200E48004E490F03CF0A3F022EDF09004
:1030F000F0AAE0FEA3E0FFC322788E7CF07D017B86
:10310000FF7A0079087E007F141229E1E490F0A292
:10311000124285F0A3124285F07F0B123885EF60D2
:1031200051122FE37F0B122FEA90F02CF090F099C0
:10313000E090F02BF090F09AE090F02AF090F09B65
:10314000E090F029F090F09CE090F030F090F09D4D
:10315000E090F02FF090F09EE090F02EF090F09F35
:10316000E090F02DF07F0B12384F7B017AF0792937
:10317000B1B07F0D123885EF600E122FE37F0D7115
:10318000EC7F0D12384FD2037F07123885EF7002A3
:103190004163122FE37F07122FEA90F00BF090F0BB
:1031A00099E090F00AF090F09AE090F009F090F039
:1031B0009BE090F008F090F09CE090F00FF090F021
:1031C0009DE090F00EF090F09EE090F00DF090F009
:1031D0009FE090F00CF07F0712384F90F018E00459
:1031E000F090F00CE090F046F090F0091242D99087
:1031F000F008124257D31226C950031242EE12426F
:10320000B81242487D3CF1E790F04312423AF1E5B2
:1032100090F04111ED941EEE940090F04040057442
:103220001EF08002EFF090F00B1242D990F00A12DB
:103230004257C31226C950031242EE1242B812423C
:10324000487D3CF1E790F05012423AF1E590F04EA3
:1032500011ED941EEE940090F04D4005741EF08028
:1032600002EFF07B017AF07931123A873000026187
:1032700040D2007B017AF0792171967F09716390C9
:10328000F0EAEFF07F0A716390F0E8715F90F0E789
:10329000715F90F0EBEFF07F0C716390F0E9EFF06D
:1032A00012403990F07DE0FF90F018E06F7039C265
:1032B0000290F06EE04401F0E04402F090F06DE026
:1032C0004440F0E04480F0A3E04404F0E04410F017
:1032D000E04420F0E04408F03003177B017AF079F5
:1032E0006D7F0A123A05800AD20290F018E090F041
:1032F0007DF0124098A292E43354011242AF54FE82
:10330000FDEC124278A294B3E433540125E0FFE4CB
:1033100033FE1242B054FD124275A202E4FE335451
:10332000017802C333CE33CED8F91242AF54FB1228
:10333000427530030B7B017AF079E67F0C123A0577
:1033400090F05CE0FF64406005EF6480701090F0E6
:103350005CE090F053F0122B89E490F05CF022EFE7
:10336000F07F0BAD07124170AF05F1CA1241517FDA
:10337000A3F1CA1241FFC2041241D4C205718B00ED
:10338000D205F1EE0000000000D205E4F5B243865C
:1033900008A2059283227F087163F1D6EF1225FD02
:1033A0007F077163EF541FFFF1D6900001EF1226E3
:1033B0000F7F051242E4900002EF12260F7F0412E5
:1033C00042E4900003EF12260F7F067163EF54076B
:1033D00090000412260F7F03F1D0900005EF122613
:1033E0000F7F02F1D0900006EF02260F123B5DE541
:1033F000D820E1FBC0D9C0DAC0DBC0DCC0DDC0DE54
:103400001242982400123845E4F5D8E5D820E1FBB3
:10341000B1A4E5DE1225FD1242982404123845E4D9
:10342000F5D8E5D820E1FBB1A490000DE5DB12262C
:103430000F90000CE5DC12260F90000BE5DD122644
:103440000F90000AE5DE12260F75D804E4F5D8E5E2
:10345000D820E1FBB1A4900011E5DB12260F90000B
:1034600010E5DC12260F90000FE5DD12260F90000C
:103470000EE5DE12260F90F0ACE012383FE4F5D8EE
:10348000E5D820E1FBE5DC30E30F90F0ADF1F62468
:10349000011242D244081225FD1242F9E5D820E17A
:1034A000FBE5DE30E554B1A4900005E5DB12260F04
:1034B000900004E5DC12260F90000312428E90006B
:1034C0000212260F123B561242F9E5D820E1FBB159
:1034D000A4900009E5DB12260F900008E5DC122617
:1034E0000F90000712428E90000612260FE9240169
:1034F0001242D244041225FD806D12430AB1A490F9
:103500000005EF12429090000412260F900003E491
:1035100012260F900002E412260F9000041242C5FA
:103520002404B196900005EF1225CA123B561242B0
:10353000F9E5D820E1FB12430AB1A4900009EF128B
:10354000429090000812260F900007E412260F9078
:103550000006E412260F9000081242C52408B19616
:10356000900009EF1225CA1242982402123845E44D
:10357000F5D8E5D820E1FBB1A4900013E5DD1226D3
:103580000F900012E5DE12260FD0DED0DDD0DCD0A9
:10359000DBD0DAD0D922F9E43AFA12258413135495
:1035A0003F1225FD90F0ADE0FBA3E0FAA3E0F92285
:1035B00090F0AF123B63E4A3F078B37CF07D017B25
:1035C000FF7A00791CFE7F081229E1F1F34A4B7063
:1035D00002C19E78B37CF07D0190F0AFB1A9123AA0
:1035E0008090F0B3E0FF7B63E4FDD1AEEFF0A3E0A9
:1035F000FF7B0C0DD1AEEFF0A3E0FF7B1FD1AEEF50
:10360000F0A3E0FF7B171DD1AEEFF0A3E0FF7B0638
:10361000D1AEEFF0A3E0FF7B3BD1AEEFF0A3E0FF34
:10362000D1AEEFF090F0AFB1A7122584FFD1BFADBE
:10363000077F08F1BCB1A7900001F1C2541FFD7FC4
:1036400007F1BCB1A7900002F1C2543FFD7F05F124
:10365000BCB1A7900003F1C2543FFD7F04F1BCB19F
:10366000A790000412259D5407FD7F06F1BCB1A769
:10367000900005F1C2547FFD7F03D19F7F027163EB
:10368000EF548090F0B2F090F0AFB1A7900006F147
:10369000C2547FFF90F0B2E04FFD7F02D19F22AC79
:1036A00007124170AF04F1CAAF05F1CA617BEFC3E5
:1036B0009D5003AF0522EFD39B4003AF032222EFBF
:1036C00075F00A84C454F0FEEF75F00A84E5F04EFC
:1036D000FF2290F0AF123B6378B27CF07D017BFF5C
:1036E0007A007924123A8078BA7CF07D017BFF7AE7
:1036F00000792C123A80E490F0C2F0FCF1F34A4BCE
:10370000601690F0AFA3A3E0F9123B50700D123B8E
:103710004A7008123B4470037F01227B017AF079E2
:10372000B2719690F0AFB1A7123B50FF90F0B7E0A6
:103730002F90F0BFF0E0C3943C74809480400AE086
:1037400024C4F090F0C27401F0123B4AFF90F0B52F
:10375000E02FFF90F0C2E02F90F0BDF0E0C394188E
:10376000748094804006E024E8F07C01123B44FF22
:1037700090F0B4E02F2C90F0BCF0E0C3941F748064
:1037800094804003741FF0E490F0BEF090F0BC12FF
:1037900043007F0BD19FA31243007F0AD19F7D80FE
:1037A0007F0CD19F90F0BFE0FFD1BFEF547FFD7F32
:1037B00009D19F7D027F01D19F7F0022D19F90F090
:1037C000AF2212259DFFD1BFEF221241A402417604
:1037D0007163EF547FFFEFC4540F75F00AA4FEEF3E
:1037E000540F2EFF227D18AF03AE02022631A20530
:1037F00092822290F0AFE0FBA3E0FAA3E022E4FD86
:10380000E5D820E1FBC0D9C0DAC0DBC0DCC0DDC038
:10381000DE113EE4F5D8E5D820E1FBE5DC5401708B
:103820000EF5DC75DB20117DE5D820E1FB7D01D0B4
:10383000DED0DDD0DCD0DBD0DAD0D9AF0522EF7519
:10384000F008A42407FFE5F03404F5DA8FD922E567
:10385000D820E1FBC0D9C0DAC0DBC0DCC0DDC0DEEF
:10386000113E75DC0075DB08E4117DE5D820E1FB35
:10387000D0DED0DDD0DCD0DBD0DAD0D922F5DEF559
:10388000DD75D8F122E4FDE5D820E1FBC0D9C0DA2E
:10389000C0DBC0DCC0DDC0DE113EE4F5D8E5D820D9
:1038A000E1FBE5DB30E3027D01D0DED0DDD0DCD012
:1038B000DBD0DAD0D9AF052290F0B8EFF0A3122711
:1038C0004200000000E47F707E17FDFC90F0B9120A
:1038D0004145C31226DF502A90F0B8E0FF1237FEB0
:1038E000EF701F1242A190F0B9E0FCA3F1E72401B0
:1038F000FFE43EFEE43DFDE43CFC90F0B9122736C7
:1039000080C3223003127F0611B87B017AF0790060
:103910007F0631197F0631D222E5D820E1FBC0D9DC
:10392000C0DAC0DBC0DCC0DDC0DE113EE4F5DCF592
:10393000DBF5DE75DD0875D8F1E5D820E1FB7156C1
:1039400075D8083182E5D820E1FB75D804740429C4
:10395000F9E43AFA3182E5D820E1FB75D80475D84C
:103960000475DC0075DB4075DE0075DD2075D8F16F
:10397000E5D820E1FBD0DED0DDD0DCD0DBD0DAD062
:10398000D922122716E48EDC8FDB1227167810124C
:1039900026F08EDE8FDD75D8F12290F0AAEFF0A32D
:1039A000EDF078AC7CF07D017BFF7A0079345180BA
:1039B00090F0AAE090F0AFF090F0ABE090F0AEF0B5
:1039C0007B017AF079AC7F0931197F0931D27F0907
:1039D00001B8E5D820E1FBC0D9C0DAC0DBC0DCC04B
:1039E000DDC0DE113EE4F5DCF5DB75DE0775DD20BC
:1039F00075D8F1E5D820E1FBD0DED0DDD0DCD0DB1E
:103A0000D0DAD0D922715D78B07CF07D017BFF7A6D
:103A100000790051801235A412258490F0B2F09004
:103A2000000112259D90F0B3F0714490F0B0F07158
:103A30004A90F0B1F090000412259D90F0B6F0711C
:103A40005090F0B7F090000612259D90F0B4F090E1
:103A5000000712259D90F0B5F090F0ACE0FF11B892
:103A600090F0ACE0FF7B017AF079B0311990F0ACC6
:103A7000E0FF21D278197CF07D017B017AF0794B4F
:103A80007E007F080229E190F0AC716390F0AC12E7
:103A900035A712258414601E14606B240260026135
:103AA0003C300209713D1236D25174802D90F0AC39
:103AB0001235A7E4613912422D5002804F78197CEB
:103AC000F07D01713D7E007F081228F1EF3395E013
:103AD0004F60115174713D1236D290F0AC1235A77F
:103AE0007401805590F046E0FF64016005EF6402C8
:103AF000700A90F0AC1235A77402803D90F0AC12C1
:103B000035A77401803390F046E070257B017AF090
:103B100079541235B07B017AF0793E1236D2C280E8
:103B2000D296C2B690F0AC1235A7E41225FD024041
:103B30002590F0AC1235A774021225FD227B017A84
:103B4000F0794B2290000202259D90000302259DF2
:103B500090000502259D75D80875D8082290F0AC14
:103B6000EFF0A3EBF0A3EAF0A3E9F02290F09C7150
:103B700063B153EF7002FF227FCC71A77F4ED185D6
:103B800090F09CD19E122584FF71A790F0A0E004D4
:103B9000F0700690F09FE004F0C390F0A0E0940372
:103BA000F1EF40DC7F0122AC07E4FBEBB1FD5014E8
:103BB000A803EC088003A2E713D8FB5401FAFF71B5
:103BC000C50B80E722AD07D17C7F02FE71E9AF050E
:103BD000EF3395E0FEEF64014E7002D2B57F197E9F
:103BE0000071E9D2B57F057E00D3EF9400EE94001A
:103BF00040090000EF1F70011E80EE2290F08E71D0
:103C000063E4A3F078937CF07D017BFF7A00793C3C
:103C1000FE7F051229E1E490F0D8F0A3F0A3F0B103
:103C200053EF7003FEFF227FF071A7E490F092F053
:103C300090F092E0B1FD4002A102E4FAEAB1FD4049
:103C40000281CCD1BEEF5403FF90F0D8E0FEC31345
:103C5000F0EF64027007FFB134E4F0806CEF6401B0
:103C60007007B12B7401F08060EF6002A12790F023
:103C700092E075F008A42A04FC90F091E0F9B18D6F
:103C8000E0FBECD39B4012E4FFB134E4F090F09100
:103C9000E004F0B18DECF08030ECC39B5017B136EE
:103CA000E0FF5401C43333335480FE90F0D8E04E2B
:103CB000F071C58014749329B18FE06C700BB12B37
:103CC0007401F090F091E014F00A813C90F0D8F18A
:103CD000E77803C333CE33CED8F9FF90F08E123796
:103CE000F62FF9EA3EFA90F092E07E0029F9EE3ADA
:103CF000FAED1225FDE490F0D8F090F092E004F097
:103D0000813090F0DAE004F0700690F0D9E004F031
:103D100090F091E0B18DE0600ED174C39405EE6433
:103D20008094805002811FD174FF2290F0D8E0442B
:103D300080F07F0171C590F092E075F008A42AF53B
:103D400082E435F0F583E5822498F582E58334F04A
:103D5000F58322E4FDFCD17D7FF0D18F7F28D14017
:103D6000FBEB6019C3ED9411EC64809480500E7FDE
:103D7000057E00D141FB0DBD00010C80E47FC87EB3
:103D80000071E9AF03EB7F0160027F00222493F50D
:103D900082E434F0F5832290F0C37163A3EDF0B1B7
:103DA00053EF7002FF227F5571A7E4F9E9B1FD508E
:103DB0002290F0C6E075F008A424EEF582E434F019
:103DC000F583E58229F582E43583F583E0FF71A769
:103DD0000980D97FBE71A7E490F0C7F090F0C7E0EA
:103DE000C39409748094805010D15CD19BEF12254C
:103DF000FD90F0C7E004F080E37F0122EEC3940859
:103E0000748094802290F09C7163B153EF7002FF34
:103E1000227FCC71A77FBED185D15C90F09CD19ED2
:103E2000EF1225FD90F0A0E004F0700690F09FE006
:103E300004F0C390F0A0E09409F1EF40DC7F012290
:103E4000FE71E9A2B5E43322D17C7F01D18F7F03DB
:103E5000D140FD7F1B7E0071E9AF0522E4FCFBEB46
:103E6000B1FD500DD1DB8002C333D8FC4CFC0B807C
:103E7000EEAF042290F0D9E0FEA3E022E4F5B243D5
:103E8000B120C2B52271A7E490F09FF0A3F022FE0A
:103E900071E9D2B5E4F5B253B1DF2290F0C3E0FB93
:103EA000A3E475F001122686A9F0FA22B153EF704F
:103EB00002FF227FCC71A77F4471A77F0122E4FC1F
:103EC000FBEBC3940274809480500DD1DB8002C35D
:103ED00033D8FC4CFC0B80E9AF0422D148A803EF97
:103EE000082290F0C37163A3EDF0E4FE90F0C6E009
:103EF000FD14F0ED6031D19B12258490F0C7F0E401
:103F0000FFEFB1FD50E690F0C7E0FD6E30E00AEE45
:103F10006418C3134480FE8004EEC313FEEDC31384
:103F200090F0C7F00F80DAAF062290F0B471639082
:103F3000F0C07401F0A374F0F0A374B7F07B017AC1
:103F4000F0F9B197EF7002FF227B017AF079B77D2B
:103F500008D1E290F0BFE06F60037F002290F0C0D4
:103F60001235A790000112259DFE122584FDEDFF5C
:103F700090F0B41235A7EE8FF012269C7F012290AC
:103F8000F08EEFF0A3EDF090F0997401F0A374F0CF
:103F9000F0A37490F07B017AF0F9D105EF7002FF85
:103FA000227B017AF079907D08D1E290F098E06F61
:103FB00060037F002290F0991237F624061242D255
:103FC00054FCFF1225FD90F08FE04F1225FD54E3C5
:103FD000FF1225FD90F08EE04F1225FD7B017AF057
:103FE0007994716C7F0122E0FDA3E0FEA3E02290B2
:103FF000F09FE0648094802275C43075C5F875C266
:104000003075C3F8E4F5C1D2C22275BF0175B4138F
:1040100075B50275BF03E4F5BBF5BF43A80175880C
:104020000175B30122C0BF75BF0143B40375BB9BCB
:1040300043B40475BBABD0BF2290F021E090F003F5
:10404000F090F022E090F002F090F023E090F00188
:10405000F090F024E090F000F090F025E090F00770
:10406000F090F026E090F006F090F027E090F00558
:10407000F090F04DE090F004F0023903AD07AC068B
:10408000EC1224CAE4FBFA79807843122428E4FB7A
:10409000FA7920784202222EE490F0B2F0A3F012D6
:1040A0003EACEF7002FF227F647E19123BE9E49080
:1040B000F0B0F0A3F090F1161230F290F0B1E09F62
:1040C000EE6480F890F0B0E06480985068E0FCA363
:1040D000E0FD25E0FFEC3138E4F0A3F074DC2FF9CB
:1040E00074F03EFA7B01123F2A90F0B1E025E0FF28
:1040F00090F0B0E03138E0FEA3E0FF117C90F0AC2E
:10410000122736E4FFFE7D207C4190F0AC31451251
:10411000231F12250390F0B2EEF0A3EFF090F0EC25
:10412000EEF0A3EFF090F0B1E004F0700690F0B084
:10413000E004F080807F012233FE74DC2FF582746E
:10414000F03EF58322E0F8A3E0F9A3E0FAA3E0FB58
:1041500022D20512338B00D2051237EE0000000088
:1041600000C20512338B0000000000C2050237EECA
:1041700031517FA231A4D20512338B000000000020
:10418000D2051237EEE4F5B25386F70000000000C6
:1041900030830AC2051237EE12337BC322C20512E6
:1041A00037EED322E4FE123DFC5028EF30E704D274
:1041B000058002C20512338B0000000000D20512F8
:1041C00037EEEF25E0FF0000000000C2051237EED9
:1041D0000E80D322300404C2058002D20512338B34
:1041E0000000000000D2051237EE0000000000C2FF
:1041F000051237EED20512338B000000000022E4D6
:10420000F5B25386F7FE123DFC5021D2051237EE6F
:104210000000000000EF25E0FF3083034401FFC2EF
:10422000051237EE00000000000E80DA227F011236
:104230003363EF5408C36001D322EDF090F0A8E09F
:10424000FAA3E0FB7C007D18FFAE02122631A3EE3C
:10425000F0A3EFF07C0022E02FFFE43E90F0A6F008
:10426000A3EFF090F0A6E0FEA3E0FFE4FCFD7BC02E
:104270007AA8F9F822FDEC4EFEED4FFF90F0E6EE45
:10428000F0A3EFF022F0A3F0A3F0A3F0A322E5DD6A
:1042900012260FE5DE541F2290F0ACE075F008A462
:1042A00022C2AF438F0143BB02538FFED2AF22FF26
:1042B00090F0E6E0FCA3E02290F0A6E0FAA3E0FB99
:1042C0007C007D3C2212259D5403C4333354C0FF2F
:1042D000E922F9E43AFA022584E0FFE4FCFDFE78E5
:1042E00008022703123363EF543FFF0237D690F0E2
:1042F000A674A8F0A374C0F02275D808E4F5D822FB
:10430000E0FF1236BFEF543FFD22E5DD54FC1313EE
:04431000543FFF22F5
:00000001FF
